:100000000C94DE000C9406010C9406010C9406017D
:100010000C9406010C9406010C9406010C94060144
:100020000C9406010C9406010C944A150C94F415DA
:100030000C9403150C9406010C9406010C94060113
:100040000C94B9140C9406010C9487140C9461144C
:100050000C9406010C9406010C9406010C94060104
:100060000C9406010C940601465335206F6E004631
:100070005335206F666600465334206F6E0046533A
:1000800034206F666600434334206F6E004343366E
:10009000206F666600434335206F6E004343352072
:1000A0006F666600434334206F6E00434334206F15
:1000B000666600544150000D0A0000000000240054
:1000C00027002A0000000000250028002B00000067
:1000D000000023002600290004040404040404048E
:1000E00002020202020203030303030301020408E3
:1000F0001020408001020408102001020408102092
:1001000000000008000201000003040700000000D6
:10011000000000006C6F6E67707265737374696DB8
:10012000656F7574006578697474756E6572616E5B
:1001300079627574746F6E006D6178627269676858
:10014000746E657373006D6964696368616E6E6572
:100150006C00736E617073686F74746170656E614A
:10016000626C656400707265736574746170656E4D
:1001700061626C656400746872750068656C70001B
:10018000666163746F727972657365740073686F0A
:100190007776616C756573000D0A00436F6D6D6154
:1001A0006E64204E4F5420666F756E642E2054721C
:1001B000792068656C703F00AD16D42111241FBEF4
:1001C000CFEFD8E0DEBFCDBF13E0A0E0B1E0EAE9B9
:1001D000F9E402C005900D92A237B107D9F728E0E3
:1001E000A2E7B3E001C01D92A833B207E1F710E027
:1001F000CDEDD0E004C02197FE010E94BA24CC3D91
:10020000D107C9F70E9464170C94C0240C94000015
:10021000E0915A07F0915B07309719F085E997E074
:10022000099580919607823F09F4BAC090F5803C09
:1002300009F499C0B8F4803909F44FC040F4E09152
:100240005E07F0915F07803809F44BC00895803A4B
:1002500009F484C0E0916407F0916507803B09F4DC
:1002600040C00895803E09F462C040F4E091680700
:10027000F0916907803D09F47AC00895803F09F440
:100280007DC0E0916E07F0916F07813F09F49BC03C
:1002900008958A3FC1F1A8F4863F09F499C040F45B
:1002A000E0917207F0917307833F09F48CC00895C1
:1002B000883F09F1E0917A07F0917B07893FF9F0D7
:1002C00008958C3F51F120F18E3F61F1E09182075A
:1002D000F09183078F3F99F00895E0916007F091C6
:1002E0006107309709F479C04091980760919707AA
:1002F000809195070994E0917607F0917707309700
:1003000009F46BC00994E0917807F0917907F7CF71
:10031000E0917C07F0917D07F2CFE0917E07F091AC
:100320007F07EDCFE0918007F0918107E8CFE09162
:100330006A07F0916B07309709F44FC060919807F6
:1003400020E8629FB001112460787F738091970745
:100350008F77682B7052809195070994E09162071E
:10036000F0916307BECFE0916607F0916707309781
:10037000A1F160919707809195070994E0916C072E
:10038000F0916D07309749F1609197077091980748
:100390006138710510F060E870E089E997E0099430
:1003A000E0917007F09171073097B9F0809198074C
:1003B00020E8829FC001112480789F7320919707C5
:1003C0002F77822B0994309741F0809197070994F9
:1003D000E0917407F091750792CF0895AF92BF92A4
:1003E000CF92DF92EF92FF920F931F93CF93DF9301
:1003F0006C017B018B01040F151FEB015E01AE1830
:10040000BF08C017D10759F06991D601ED91FC9151
:100410000190F081E02DC6010995892B79F7C5017E
:10042000DF91CF911F910F91FF90EF90DF90CF90D0
:10043000BF90AF900895FC01538D448D252F30E07F
:10044000842F90E0821B930B541710F0CF960895E1
:1004500001970895FC01918D828D981761F0A28D0E
:10046000AE0FBF2FB11D5D968C91928D9F5F9F73D4
:10047000928F90E008958FEF9FEF0895FC01918D8A
:10048000828D981731F0828DE80FF11D858D90E0F7
:1004900008958FEF9FEF0895FC01918D228D892F94
:1004A00090E0805C9F4F821B91098F73992708957C
:1004B0008BE796E00E944C0221E0892B09F420E0B2
:1004C000822F089580E090E0892B29F00E94580245
:1004D00081110C9400000895FC01A48DA80FB92F80
:1004E000B11DA35ABF4F2C91848D90E001968F735C
:1004F0009927848FA689B7892C93A089B1898C917B
:10050000837080648C93938D848D981306C00288C9
:10051000F389E02D80818F7D80830895EF92FF9293
:100520000F931F93CF93DF93EC0181E0888F9B8D16
:100530008C8D98131AC0E889F989808185FF15C0D0
:100540009FB7F894EE89FF896083E889F9898081F3
:100550008370806480839FBF81E090E0DF91CF91C2
:100560001F910F91FF90EF900895F62E0B8D10E0E4
:100570000F5F1F4F0F731127E02E8C8D8E110CC053
:100580000FB607FCFACFE889F989808185FFF5CF9E
:10059000CE010E946C02F1CFEB8DEC0FFD2FF11D0F
:1005A000E35AFF4FF0829FB7F8940B8FEA89FB89DB
:1005B00080818062CFCFCF93DF93EC01888D882339
:1005C000B9F0AA89BB89E889F9898C9185FD03C0B6
:1005D000808186FD0DC00FB607FCF7CF8C9185FF9B
:1005E000F2CF808185FFEDCFCE010E946C02E9CF72
:1005F000DF91CF910895833081F028F4813099F014
:100600008230A9F008958730A9F08830C9F084308D
:10061000B1F4809180008F7D03C0809180008F773E
:1006200080938000089584B58F7784BD089584B544
:100630008F7DFBCF8091B0008F778093B0000895BD
:100640008091B0008F7DF9CFCF93DF93282F30E0DA
:10065000F901E050FF4F8491F901E451FF4FD4912B
:10066000F901E852FF4FC491CC23A1F081110E94FF
:10067000FB02EC2FF0E0EE0FFF1FE253FF4FA591BE
:10068000B491EC91ED2381E090E009F480E0DF91FA
:10069000CF91089580E090E0FACF1F93CF93DF933E
:1006A000282F30E0F901E050FF4F8491F901E45127
:1006B000FF4FD491F901E852FF4FC491CC23A9F028
:1006C000162F81110E94FB02EC2FF0E0EE0FFF1FAE
:1006D000EC53FF4FA591B4918FB7F894EC911111A1
:1006E00008C0D095DE23DC938FBFDF91CF911F919F
:1006F0000895DE2BF8CFCF93DF9390E0FC01E45117
:10070000FF4F249188529F4FFC0184918823C9F0A8
:1007100090E0880F991FFC01E654FF4FA591B4911A
:10072000FC01EC53FF4FC591D49161110DC09FB7EF
:10073000F8948C91209582238C9388812823288398
:100740009FBFDF91CF910895623051F49FB7F89425
:100750003C91822F809583238C93E8812E2BEFCFC1
:100760008FB7F894EC912E2B2C938FBFEACF1F9369
:10077000CF93DF93182FEB0161E00E947B0320975A
:1007800039F460E0812FDF91CF911F910C944D03DC
:10079000CF3FD10511F461E0F5CFE12FF0E0E0505B
:1007A000FF4FE491E33031F140F4E130B1F0E23059
:1007B000E1F0C038D1057CF7E4CFE73029F1E8302B
:1007C00059F1E430B1F7809180008062809380001D
:1007D000D0938B00C0938A0004C084B5806884BD28
:1007E000C7BDDF91CF911F91089584B5806284BD0C
:1007F000C8BDF7CF80918000806880938000D0933F
:100800008900C0938800EDCF8091B000806880930C
:10081000B000C093B300E5CF8091B00080628093B8
:10082000B000C093B400DDCF3FB7F894809140048E
:1008300090914104A0914204B091430426B5A89B35
:1008400005C02F3F19F00196A11DB11D3FBFBA2F62
:10085000A92F982F8827BC01CD01620F711D811D22
:10086000911D42E0660F771F881F991F4A95D1F7A7
:1008700008958F929F92AF92BF92CF92DF92EF92A4
:10088000FF924B015C010E9414046B017C010E94E9
:1008900014046C197D098E099F09683E7340810517
:1008A0009105A8F321E0821A9108A108B10888EE09
:1008B000C80E83E0D81EE11CF11C81149104A10430
:1008C000B10429F7FF90EF90DF90CF90BF90AF90E9
:1008D0009F908F9008952FB7F89460913C04709189
:1008E0003D0480913E0490913F042FBF0895CF9224
:1008F000DF92EF92FF920F931F93CF93DF93EC0160
:1009000088810E9424038C010E946B042889398904
:100910002017310731F06A8B7B8B8C8B9D8B198B69
:10092000088BCA88DB88EC88FD886C197D098E09E4
:100930009F09CA80DB80EC80FD806C157D058E05EB
:100940009F0530F08E859F859D878C871F870E873A
:100950002C853D858E859F852817390781F04A852E
:100960005B8542305105A1F48E819F81A885B985B0
:100970000196A11DB11D8E839F83A887B987DF9142
:10098000CF911F910F91FF90EF90DF90CF9008953E
:100990004115510531F42130310589F7892B21F3B7
:1009A000EECF4130510559F7232B49F7019739F71D
:1009B000DBCF50914F0440914E04852F90E0242FBF
:1009C00030E0541718F0821B930B0895805B9F4F03
:1009D000FACF80914F04E0914E048E1751F0EF5FF3
:1009E000E03508F0E0E0F0E0E551FC4F808190E078
:1009F00008958FEF9FEF089580914F0490914E04DA
:100A0000891769F09F5F903508F090E0E92FF0E0DA
:100A1000E551FC4F808190934E0490E008958FEF54
:100A20009FEF08950F931F93CF93DF93FC014081B5
:100A3000518162817381452B462B472BB9F0EC0124
:100A40000E946B040C811D812E813F81AB01BC0192
:100A5000401B510B620B730B81E0088119812A81C5
:100A60003B81401751076207730708F480E0DF916C
:100A7000CF911F910F910895CF93DF93EC010E94C6
:100A80006B046C837D838E839F83DF91CF91089568
:100A9000AF92BF92CF92DF92EF92FF920F931F938C
:100AA000CF93DF93EC018B017A01E1E0F0E0CE011E
:100AB000BF010E9470246017710788F4D12CC12CEB
:100AC0003097B1F4F9011082DF91CF911F910F910E
:100AD000FF90EF90DF90CF90BF90AF900895CF013F
:100AE000809FF001819FF00D909FF00D1124DFCFCA
:100AF000CE01BF010E947024462FA62EB72EEC0116
:100B0000CF01B8010E947024FB01C114D10479F413
:100B10001A141B0464F0309799F660E3640FD9014E
:100B20006C93BFEFCB1ADB0A2F5F3F4FC9CF9AE020
:100B3000A916B10494F367E5E114F10479F367E3CE
:100B4000EDCF90914506992339F0E0915504F0914D
:100B50005604309709F009940895FF920F931F935C
:100B6000CF93DF9330E2F32E662311F020E3F22ED1
:100B70008A01FA01219121110BC0EC011C161D06FE
:100B800054F48F2D0E94A1052197F8CF0197F2CF41
:100B900018161906DCF3F80181918F01811106C046
:100BA000DF91CF911F910F91FF9008950E94A105B1
:100BB000F2CFCF93DF93EC01FE018491219688233D
:100BC00019F00E94A105F8CFDF91CF910895CF933E
:100BD000DF93EC018991811106C087EB90E0DF91F2
:100BE000CF910C94D9050E94A105F4CFE7E5F4E07C
:100BF00030E020E040815181452B21F44281538136
:100C0000452B41F02F5F3F4F34962436310591F745
:100C100080E00895220F331F220F331FF901E95A94
:100C2000FB4F918380837383628381E0089587FF04
:100C30000AC09CE0980F923030F08D3F21F0803F49
:100C400018F4807F089580E00895982F9F7E282FC4
:100C50002F7C203839F0803E29F081E0903C19F05B
:100C600080E0089581E00895DC018D919C91DC0184
:100C7000ED91FC910190F081E02D09941F93CF93A9
:100C8000DF932150203118F587FF21C0D42F162F74
:100C9000C82F622F682B80918407909185070E944E
:100CA0003406612F6F7780918407909185070E94A9
:100CB0003406CF7EC03C59F06D2F6F77809184074A
:100CC00090918507DF91CF911F910C943406DF91AD
:100CD000CF911F910895242F462F682F80EB0C94FD
:100CE0003E066D3F48F46A3F10F4683F39F4FC015A
:100CF000808191810C9434066E3FC8F70895813E3F
:100D000010F40C943E06883F28F0682F84E897E0A2
:100D10000C947106089580914E0690914F060497A9
:100D200009F580919E036FEF70E0811102C06CE0C5
:100D300070E085E00E94B70380919F036FEF70E041
:100D4000811102C06CE070E086E00E94B7038091E0
:100D5000A0036CE070E0882311F06FEF70E08BE08F
:100D60000C94B703089580914904EFEFE80FE83041
:100D700048F410929D0380919C03882351F08130A8
:100D800019F1089589508830B0F781E080939D0370
:100D9000F2CF809148046FEF70E0811102C06CE0E7
:100DA00070E085E00E94B703809144046CE070E03D
:100DB000882311F06FEF70E086E00E94B70370E0C7
:100DC00060E08BE00C94B703E03108F074C0F0E011
:100DD000E451F94F0C94BA24FC060B0713071D07C6
:100DE00027072C07310736073B073F07430747070D
:100DF0004B074F075307570710929D0370E060E0C1
:100E000085E00E94B70370E060E086E00E94B703CF
:100E10006FEF70E0D6CF10929D0370E060E085E048
:100E20000E94B703C7CF10929D0370E060E085E099
:100E30000E94B7036FEF70E0E8CF10929D036FEF51
:100E400070E085E00E94B70370E060E0B5CF1092DB
:100E50009D036FEF70E0D4CF10929D036FEF70E0B1
:100E6000DECF10929D036FEF70E0E1CF10929D03F3
:100E700070E060E0E6CF81E080939D03BFCF81E02A
:100E800080939D03CACF81E080939D03CECF81E004
:100E900080939D03D4CF81E080939D03DACF81E0DE
:100EA00080939D03DBCF81E080939D03DCCF81E0C5
:100EB00080939D03DDCF08954091490460E088E46C
:100EC0000C946B06409149046FE788E40C946B0620
:100ED0001092710610926C061092670610926206CC
:100EE0001092610610925E0610925C0610926006E7
:100EF00010925D0610925B0610925A0610925F06E1
:100F000008959091900380919103811115C09111E2
:100F10002BC080918F036CE070E0811126C06FEFD1
:100F200070E085E00E94B7036FEF70E086E00E94FA
:100F3000B7036FEF70E012C080918F03911111C061
:100F4000811112C06FEF70E085E00E94B7036CE082
:100F500070E086E00E94B7036CE070E08BE00C94D8
:100F6000B7036FEF70E08111089585E00E94B70329
:100F70006CE070E0DBCF80914E0690914F0682309E
:100F8000910509F442C068F5009779F10197B1F134
:100F90008091000190918C03992309F444C0823020
:100FA000D1F18330E1F1813029F470E060E085E037
:100FB0000E94B7038091040190910501A091060160
:100FC000B09107018093500690935106A09352066A
:100FD000B093530680E596E00E943C0510928C0386
:100FE00008950597A8F68FEF06C0809147048823DF
:100FF000D1F38091010180930001CACF8091460412
:10100000882389F380910201F6CF80918D038111AD
:10101000EACF83E0F0CF70E060E086E0C9CF70E017
:1010200060E08BE0C5CF823009F1833019F1813067
:1010300029F46AE570E085E00E94B703809104011D
:1010400090910501A0910601B0910701809350068F
:1010500090935106A0935206B093530680E596E014
:101060000E943C0581E080938C0308956AE570E05E
:1010700086E0E2CF6AE570E08BE0DECF80914E063D
:1010800090914F060297B1F4809188036CE070E074
:10109000882311F06FEF70E085E00E94B703809124
:1010A00089036CE070E0882311F06FEF70E086E058
:1010B0000C94B703089580914E0690914F060297C5
:1010C00039F40E943E086CE070E08BE00C94B703AA
:1010D0000895682F8BE796E00C948E02CF93DF93F0
:1010E000EC018BE796E00E944C02009739F08BE709
:1010F00096E00E942A02888381E090E0DF91CF9100
:10110000089580918B0391E0892780938B03409110
:1011100049046FE784E40C946B0680914D048111BF
:10112000FCCF089580914C048F5F843408F080E0F8
:1011300090914B049817E1F32FB7F89490914D04D8
:10114000992359F0E82FF0E0EF55FC4F608380932E
:101150004C042FBF81E090E0089581E080934D041E
:101160006093E6031092E50382E086BB80916F00F6
:10117000826080936F00809180008F7B8068809375
:101180008000809184009091850040969093890022
:1011900080938800DECF90E080E0089580918E03F8
:1011A000882341F180919C0361E08823D1F0813054
:1011B00089F480919D0360E0811113C061E08EE0AD
:1011C0000E944D0361E08FE00E944D0360E080E1EA
:1011D0000E944D0386E496E00E943C0510928E0327
:1011E00008958EE00E944D0361E08FE00E944D0360
:1011F00061E0EDCF60E08EE00E944D0360E08FE0A3
:101200000E944D0360E080E10E944D0386E496E079
:101210000E943C0581E080938E0308956CE070E0AD
:1012200085E00E94B7036CE070E086E00E94B7039F
:101230006CE070E08BE00C94B703CF9380914E0686
:1012400090914F060197C1F5C0910201C130D9F4C8
:101250006FEF70E085E00E94B7036CE070E086E01D
:101260000E94B7036CE070E08BE00E94B7038091AE
:101270004604882309F1C150C330F0F40E940E09DE
:10128000CF910C94BB07C23041F46CE070E085E074
:101290000E94B7036FEF70E0E2CFC33041F76CE01C
:1012A00070E085E00E94B7036CE070E086E00E9489
:1012B000B7036FEF70E0D8CFCF9108954091490404
:1012C000682F85E40E946B060C941D09CF938091D2
:1012D0004E0690914F06892BE1F5C09101016FEF09
:1012E00070E0C13081F1C23069F46CE070E085E0FB
:1012F0000E94B7036FEF70E086E00E94B7036CE0D6
:1013000070E00EC0C330D9F46CE070E085E00E945C
:10131000B7036CE070E086E00E94B7036FEF70E007
:101320008BE00E94B70380914704882391F0C1505D
:10133000C33078F40E940E09CF910C94BB07CF3FC5
:1013400091F76CE070E085E00E94B7036CE070E01C
:10135000D3CFCF910895FC0101900020E9F7319798
:10136000AF01481B590BBC018BE796E00C94EE01D2
:101370008F929F92AF92BF920F931F93CF93DF9361
:10138000CDB7DEB7A1970FB6F894DEBF0FBECDBFC5
:1013900019A2423008F44AE08E010F5D1F4F842EDF
:1013A000912CB12CA12CA50194010E949824E62F28
:1013B000B901CA01EA30F4F4E05DD801EE938D0181
:1013C000232B242B252B79F790E080E0109719F040
:1013D000CD010E94AB09A1960FB6F894DEBF0FBEF7
:1013E000CDBFDF91CF911F910F91BF90AF909F9094
:1013F0008F900895E95CE1CF0F931F93CF93DF9314
:101400008C01D0E0C0E0F801EC0FFD1F6491662371
:1014100041F08BE796E00E948E02892B11F0219615
:10142000F2CF83EF92E00E94AB098C0F9D1FDF91FA
:10143000CF911F910F910895CF92DF92EF92FF927B
:101440000F931F930E946B040091940310919503D6
:1014500020919603309197036B017C01C01AD10A49
:10146000E20AF30A97018601093B4BE014072105C4
:10147000310508F064C00093040110930501209326
:101480000601309307016093940370939503809352
:101490009603909397034AE0C701B6010E94B809EA
:1014A00083EF92E00E94AB098091040190910501C5
:1014B000A0910601B0910701B695A79597958795DC
:1014C0008D3D25E09207A105B10520F08CED95E05A
:1014D000A0E0B0E08D379105A105B10520F48DE7BE
:1014E00090E0A0E0B0E08093040190930501A09308
:1014F0000601B09307018091040190910501A0912C
:101500000601B09107018093500690935106A09375
:101510005206B093530680E596E00E943C05409148
:1015200049046FE780E40E946B0683EB90E01F9113
:101530000F91FF90EF90DF90CF900C94FC09609397
:101540009403709395038093960390939703D3CF5E
:10155000CF93803109F066C06430C9F4403488F418
:1015600010929E038BEA90E00E94FC0980914E0647
:1015700090914F068430910509F04FC0CF910C94A3
:101580008B0681E080939E0384EA90E0EDCF653086
:1015900069F4403428F410929F038CE990E0E4CF82
:1015A00081E080939F0385E990E0DECF663069F4A7
:1015B000403428F41092A0038DE890E0D5CF81E06C
:1015C0008093A00386E890E0CFCF6431B1F440343B
:1015D00050F4109288038EE790E00E94FC0981E0AD
:1015E00080938A03C3CFC1E0C093880387E790E06C
:1015F0000E94FC09C0938A03B9CF653109F0B6CFC8
:10160000403428F4109289038FE690E0E6CFC1E0E1
:10161000C093890388E690E0EBCF029719F4CF914D
:101620000C945B08CF910895CF92DF92EF92FF92D6
:101630000E941404C0908403D0908503E090860338
:10164000F09087036C197D098E099F090E944C2335
:101650006B017C0120E034E244EF57E40E94DA237E
:1016600018163CF4C12C44E2D42E44EFE42E47E497
:10167000F42E6091820370918303072E000C880B77
:10168000990B0E944E23A70196010E9438229B01CC
:10169000AC0160E074E284E799E40E94A42220E0B7
:1016A00030E040EC51E40E94A42220E030E040E72A
:1016B00052E40E94DF230E9416236B017093810382
:1016C0006093800380917E0390917F038B3A910514
:1016D0000CF461C087E390E09093830380938203CE
:1016E0000E9414046093840370938503809386039F
:1016F0009093870380917C0390917D0384309105C2
:101700000CF062C0FC01EE0FFF1FEC58FC4FD182C1
:10171000C082019690937D0380937C0310927303A3
:101720001092720360917E0370917F03072E000C6C
:10173000880B990B0E944E239B01AC0160E070E086
:1017400080EF91E40E94A42220E030E04AE754E4D4
:101750000E94DF230E941D236115710581059105FB
:1017600009F47EC0DC01CB018D3D25E09207A10587
:10177000B10520F08CED95E0A0E0B0E0809304018D
:1017800090930501A0930601B0930701FF90EF909D
:10179000DF90CF9008959C012759310924313105FC
:1017A00018F484E190E098CF9C012358310924314A
:1017B000310518F48FE090E08FCF8238910509F45D
:1017C0008FCF8CE99FEF88CF049709F0ABCF1092B1
:1017D0007D0310927C03809172039091730320919A
:1017E000740330917503820F931F2091760330911B
:1017F0007703820F931F2091780330917903820F32
:10180000931F20917A0330917B03820F931F909353
:1018100073038093720397FD03969595879595952D
:1018200087958D3221E0920714F08CE291E08431AB
:10183000910514F484E190E090937F0380937E03FC
:10184000609104017091050180910601909107015A
:101850004AE00E94B80983EF92E00E94AB0962CF90
:1018600081E090E0A0E0B0E089CF2F923F924F92CC
:101870005F926F927F928F929F92AF92BF92CF9220
:10188000DF92EF92FF920F931F93CF93DF93CDB729
:10189000DEB72C970FB6F894DEBF0FBECDBFFE01AA
:1018A000B196E190F1908F019E012F5F3F4F59015A
:1018B0008DE2282E2E0132E0430E511C9AE0392E83
:1018C000F7018081882339F1853231F09FEFE91AE1
:1018D000F90A0E94A105F4CFF70181818033A1F1BB
:1018E000F2E0EF0EF11C912C90ED980FF701D12C46
:1018F000C12C9A3008F446C0D12CC12C833609F48F
:101900009CC00CF057C0853209F4AEC0883509F48C
:1019100079C08111D5CF2C960FB6F894DEBF0FBEDB
:10192000CDBFDF91CF911F910F91FF90EF90DF908E
:10193000CF90BF90AF909F908F907F906F905F906F
:101940004F903F902F900895828197012D5F3F4FD8
:10195000790199249394C8CF9FE9980F9630F0F4B9
:10196000282F082E000C330B275531092B30310559
:101970002CF63C9CC0013D9C900D11246C01C20EC4
:10198000D31E81917F0190ED980F9A3028F7082E91
:10199000000C990B9C0120533109EBCF9FEB980F62
:1019A000963008F0ABCF282F082E000C330B2753AE
:1019B0003109DCCF833709F44AC0FCF4843609F0DE
:1019C0007FCF3801F2E06F0E711CF80180819181A8
:1019D000950197FF05C09195819591092982920102
:1019E00050E040E06AE070E00E944805A501692DE2
:1019F000C6010E94AD05830163CF853789F0883722
:101A000009F05ECF3801F2E06F0E711C41E050E04A
:101A1000883511F050E040E0950160E170E009C0C8
:101A2000380132E0630E711C950150E040E06AE03D
:101A300070E0F80180819181D7CF6801F2E0CF0E8C
:101A4000D11CF80180810E94A105860139CF48018F
:101A5000F2E08F0E911CF8014081518160E0C601D7
:101A60000E94AD0584012CCF85E233CFCF93DF9365
:101A7000CCE2D1E0DF93CF930E94350C80914904F2
:101A80001F928F938CE491E09F938F930E94350C6B
:101A9000809148041F928F938FE591E09F938F93DD
:101AA0000E94350C809147041F928F938BE691E042
:101AB0009F938F930E94350C809146041F928F93C1
:101AC00083E891E09F938F930E94350C80914404AA
:101AD0001F928F938DE991E09F938F930E94350C15
:101AE000809159068F93809158068F9387EB91E0F0
:101AF0009F938F930E94350CDF93CF930E94350CF8
:101B00008DB79EB74C960FB6F8949EBF0FBE8DBF93
:101B1000DF91CF910895CF93DF93CCE2D1E0DF93B3
:101B2000CF930E94350C8FEC91E00E94AB0983EFBC
:101B300092E00E94AB098BEE91E09F938F930E94FD
:101B4000350CDF93CF930E94350C83E092E09F9396
:101B50008F930E94350C83EF92E09F938F930E94A6
:101B6000350C89E192E09F938F930E94350C86E2B9
:101B700092E09F938F930E94350C8BE392E09F93AA
:101B80008F930E94350C88E492E09F938F930E947C
:101B9000350C86E692E09F938F930E94350C8FE779
:101BA00092E09F938F930E94350C8AE992E09F9375
:101BB0008F930E94350C85EB92E09F938F930E9448
:101BC000350CDF93CF930E94350C8DB79EB74C96A2
:101BD0000FB6F8949EBF0FBE8DBFDF91CF910895D1
:101BE00084EC92E09F938F930E94350C0F900F909E
:101BF00008958FEE92E09F938F930E94350C0F9083
:101C00000F90089520910301922F990F920F9450F5
:101C1000890F80934A04909100011F929F931F9215
:101C20008F9386EF92E09F938F930E94350C0E94D2
:101C30006609109299032091490440E060914A049A
:101C400080EC0E943E0610929B030F900F900F9025
:101C50000F900F900F9008951F93CF93DF93EC0197
:101C6000162F0E942122181739F0612FCE01DF9123
:101C7000CF911F910C942922DF91CF911F9108954C
:101C800010929B0360919A036093030181E090E0BE
:101C90000E942C0E10929903809198038093010169
:101CA0000E94660984E193E00E94AB0983EF92E011
:101CB0000E94AB09809103011F928F938AE293E007
:101CC0009F938F930E94350C0F900F900F900F9061
:101CD0000895CF93DF93D82F80919B03811103C088
:101CE00081E080939B03C09103018091990381114E
:101CF00009C0C0939A0381E0809399038091010108
:101D0000809398038FEF809301016FEF70E085E07F
:101D10000E94B7036FEF70E086E00E94B7036FEF99
:101D200070E08BE00E94B703D1110CC08AE2C13091
:101D300061F068F0C150C093030109C0CA3238F4A1
:101D4000CF5FF9CFCA32D1F781E080930301609170
:101D5000030181E090E00E942C0E809103011F920C
:101D60008F9384E393E09F938F930E94350C0F90A1
:101D70000F900F900F90DF91CF91089560914E06D4
:101D800090E080E00C942C0E80914E0690914F06CE
:101D9000909393038093920384E090E090934F0696
:101DA00080934E0661E08EE00E944D0361E08FE07B
:101DB0000E944D0360E080E10E944D030E948B066B
:101DC0000C94BE0E80914E0690914F069093930313
:101DD0008093920382E090E090934F0680934E06AA
:101DE00061E08EE00E944D0360E08FE00E944D03B1
:101DF00061E080E10E944D030E945B080C94BE0EDE
:101E000080914E0690914F06909393038093920396
:101E100081E090E090934F0680934E0660E08EE064
:101E20000E944D0361E08FE00E944D0360E080E17D
:101E30000E944D030E941D090C94BE0E80914E0617
:101E400090914F06909393038093920310924F06C4
:101E500010924E0661E08EE00E944D0360E08FE03C
:101E60000E944D0360E080E10E944D030E946609DC
:101E70000C94BE0ECF92DF92EF92FF9220914E060D
:101E800030914F06882309F43FC02115310551F5E3
:101E90000E94000F8FE393E00E94AB09C0904E06B2
:101EA000D0904F060D2C000CEE08FF084AE0C70149
:101EB000B601F7FE0DC06DE28BE796E00E948E0240
:101EC00066277727CB016C197D098E099F094AE0A7
:101ED0000E94B80983EF92E0FF90EF90DF90CF90DF
:101EE0000C94AB092130310519F40E94E20ED2CFD7
:101EF0002230310519F40E94C40ECCCF24303105B4
:101F000049F60E941E0FC6CF2430310571F32230EE
:101F1000310509F4BDCF2130310599F3232B09F0A8
:101F2000B9CFE9CF809192039091930381309105CD
:101F300049F030F08230910539F0049739F0089576
:101F40000C941E0F0C94000F0C94E20E0C94C40E13
:101F500080914E0690914F0683309105D1F0909379
:101F600093038093920383E090E090934F068093D5
:101F70004E0660E08EE00E944D0360E08FE00E941C
:101F80004D0361E080E10E944D030E9481070C94A3
:101F9000BE0E0C94920FCF93C82F80918B03C0314B
:101FA00011F178F4CD3091F180918B03882309F4FD
:101FB00072C080914404882309F46DC0CF910C94C1
:101FC0008108C131C9F1C43179F7882321F08091AA
:101FD000440481110EC080914E0690914F060697E1
:101FE00019F381E010C0882339F0809144048823DC
:101FF00019F00E948108D8CF80914E0690914F062B
:10200000069791F280E00E943A0FCECF882321F00C
:10201000809144048111EDCF80914E0690914F063E
:10202000069711F280919B03811103C00E94A80FB3
:10203000BBCF0E94400EB8CF882321F0809144048A
:102040008111D7CF80914E0690914F068630910531
:10205000F9F0909393038093920386E090E090933D
:102060004F0680934E068CE291E0A0E0B0E08093B2
:10207000460690934706A0934806B093490686E427
:1020800096E00E943C050E94CE080E94B3068CCFC9
:102090000E94920F89CF80914E0690914F06823018
:1020A000910509F4E9C038F4009729F1019709F482
:1020B0007FC0CF9108958430910509F426C108F4BA
:1020C00069C10697B1F780919C038111F0C1C230BC
:1020D00009F4E4C108F0D8C1C13059F7E0914804CF
:1020E0006E2F6C27609348048BE090E00E942C0ECA
:1020F000CF910C94B306C150CE30D8F6EC2FF0E05F
:10210000EC57FF4E0C94BA249210A510B110591040
:10211000C510CB10C9105910591059105910C210C0
:102120005910BD1080910101813021F081E0809330
:10213000010108C080914704882319F0CF910C94C5
:102140001C0A81E0CF910C94020E80910101823033
:1021500011F082E0ECCF809147048111EFCF82E053
:10216000F1CF80910101833011F083E0E0CF8091C5
:1021700047048111E3CF83E0E5CF80919B0388235F
:1021800009F41CCFCF910C94400E80E0CF910C94B9
:10219000690E81E0FBCF6091470481E0682760937E
:1021A00047048CE090E00E942C0ECF910C946609BD
:1021B000C150CE3008F07DCFEC2FF0E0EE51FF4E55
:1021C0000C94BA24F01010111E115910A6112F11E1
:1021D0002C11591059105910591059105910DE0F5F
:1021E00080910201813039F081E08093020180E02A
:1021F0000E945E0906C0809146048823C1F30E94B4
:102200001C0A809102011F928F9387E493E09F93B1
:102210008F930E94350C0F900F900F900F9049CF25
:1022200080910201823029F082E08093020181E0F6
:10223000DFCF809146048823D1F3E1CF8091020162
:10224000833029F083E08093020182E0D1CF809136
:1022500046048823D1F3D3CFCF910C9462076091C9
:10226000460481E06827609346048DE090E00E9478
:102270002C0ECF910C941D09C150CE3008F019CF0F
:10228000EC2FF0E0EA5BFE4E0C94BA245411671177
:102290009E105910A61178112C115910591059106F
:1022A000591059105910DE0F409149046FE784E32B
:1022B0000E946B0680918A03882331F08091880305
:1022C00091E0892780938803CF910C943E08409138
:1022D00049046FE785E30E946B0680918A03882397
:1022E00099F38091890391E0892780938903ECCF4A
:1022F00060918D0381E0682760938D0380E290E018
:102300000E942C0ECF910C945B08C33099F1A8F475
:10231000C130F9F0C23009F0CCCEC0919F0361E02A
:10232000C627C0939F030E948B066FE7C69F602D50
:1023300011244091490485E01AC0C73009F48CCFBC
:10234000CE3009F43BCEC53009F0B3CECF910C941A
:102350005C07E0919E03CE27C0939E030E948B06EC
:102360006FE7C69F602D11244091490484E0CF910E
:102370000C946B06C091A00361E0C627C093A00334
:102380000E948B066FE7C69F602D1124409149047F
:1023900086E0EDCFC931F9F0CB3109F453C0C2303A
:1023A00009F087CE409149046FE78FE30E946B06E6
:1023B00080919103882321F19091900380918F0364
:1023C000911136C081111CC010929103109290039C
:1023D00010928F0315C09091900380919103811109
:1023E00012C091110DC080918F03811119C081E03D
:1023F00080939103409149046FE78CE30E946B0640
:10240000CF910C94810780918F0391112FC081117E
:10241000F7CF81E0809390034091490460E0EDCFD5
:1024200081E0809391038093900310928F03F4CF07
:102430008111E6CF109291031092900381E0809376
:102440008F03DECF909190038091910381110CC096
:102450009111D6CF80918F03882371F010928F0352
:102460004091490460E00EC080918F038111C8CF74
:10247000109291031092900381E080938F0340911A
:1024800049046FE78DE3BACFC53009F431CEC730C8
:1024900009F00FCE81E080939C032ACE6091440422
:1024A00081E06827609344048FE190E01FCE813083
:1024B00009F0FFCDC33099F060F4C13009F0F9CDD7
:1024C00080914904823008F413CE815080934904EE
:1024D0000FCEC53059F0C73009F40ACEEACD80914D
:1024E0004904803108F004CE8F5FF0CF10929C0336
:1024F000FFCDCF93DF9390914904981336C060933A
:102500004A048BEA689F612D112466956F5F609382
:10251000030181E090E00E942C0E80910301982F2E
:10252000990F990F891B90914A049C5F890F8093A2
:102530000001809301010E94660981E080930201FD
:10254000C0914E06D0914F06C130D10511F40E94C2
:102550001D0910928A031092880310928903229712
:1025600021F4DF91CF910C945B08DF91CF91089516
:1025700061E08EE00E944D0361E08FE00E944D0318
:1025800061E080E10E944D0370E060E085E00E9420
:10259000B70370E060E086E00E94B70370E060E09F
:1025A0008BE00E94B70368EE73E080E090E00E9449
:1025B000390460E090E080E00E942C0E61E081E050
:1025C00090E00E942C0E60E082E090E00E942C0ED1
:1025D00061E08AE090E00E942C0E60E08BE090E0E9
:1025E0000E942C0E6CE384E190E00E942C0E61E0CE
:1025F0008CE090E00E942C0E61E08DE090E00E9463
:102600002C0E6FEF8EE190E00E942C0E60E08FE1C7
:1026100090E00E942C0E60E080E290E00E942C0E80
:10262000F0E0E0E009940E94B81208950C94212291
:102630008130910579F4809144041F928F938AE34D
:1026400093E09F938F930E94350C0F900F900F9003
:102650000F9008950297ECF3FB01828193810E9411
:10266000F2218A3058F081E08093440461E08FE1E8
:1026700090E00E942C0E0E94F90DEBCF0E94F00D0D
:10268000E8CF8130910579F4809145041F928F93B2
:102690008AE393E09F938F930E94350C0F900F90E5
:1026A0000F900F9008950297ECF3FB0182819381C4
:1026B0000E94F2218A3050F080934504682F8EE109
:1026C00090E00E942C0E0E94F90DECCF0E94F00DBC
:1026D000E9CF8130910579F4809149041F928F935D
:1026E0008AE393E09F938F930E94350C0F900F9095
:1026F0000F900F9008950297ECF3FB018281938174
:102700000E94F2219FEF980F903150F4809349047A
:10271000682F8AE090E00E942C0E0E94F90DEACF0B
:102720000E94F00DE7CF8130910589F48091590620
:102730008F93809158068F9381E693E09F938F93B8
:102740000E94350C0F900F900F900F9008950297F4
:10275000ECF3FB01828193810E94F2219C01285CB1
:1027600031092D3F384078F49093590680935806EC
:102770006AE070E00E94842484E190E00E942C0EC4
:102780000E94F90DE3CF0E94F00DE0CF813091055A
:1027900079F4809146041F928F938AE393E09F938C
:1027A0008F930E94350C0F900F900F900F9008950B
:1027B0000297ECF3FB01828193810E94F221823027
:1027C000A8F461E0892B09F460E0609346048CE092
:1027D00090E00E942C0E80914E0690914F0601973A
:1027E00011F40E941D090E94F90DE1CF0E94F00D25
:1027F000DECF8130910579F4809147041F928F9349
:102800008AE393E09F938F930E94350C0F900F9073
:102810000F900F9008950297ECF3FB018281938152
:102820000E94F2218230A8F461E0892B09F460E073
:10283000609347048CE090E00E942C0E80914E063D
:1028400090914F06892B11F40E9466090E94F90DA0
:10285000E1CF0E94F00DDECF8130910579F48091B7
:1028600048041F928F938AE393E09F938F930E9473
:10287000350C0F900F900F900F9008950297ECF386
:10288000FB01828193810E94F2218230B8F461E0E1
:10289000892B09F460E0609348048BE090E00E948B
:1028A0002C0E80914804882331F083E080939407B4
:1028B0000E94F90DE2CF10929407FACF0E94F00D1A
:1028C000DCCF1F920F920FB60F9211242F933F93DC
:1028D0004F935F936F937F938F939F93AF93BF9328
:1028E000EF93FF938BE796E00E946C02FF91EF91CC
:1028F000BF91AF919F918F917F916F915F914F9118
:102900003F912F910F900FBE0F901F9018951F921F
:102910000F920FB60F9211242F938F939F93EF93E3
:10292000FF93E0918B06F0918C068081E0919106F7
:10293000F091920682FD1BC09081809194068F5F7A
:102940008F7320919506821741F0E0919406F0E094
:10295000E558F94F958F80939406FF91EF919F91E1
:102960008F912F910F900FBE0F901F90189580811F
:10297000F4CF1F920F920FB60F9211242F933F9313
:102980008F939F93AF93BF9380913C0490913D04AC
:10299000A0913E04B0913F0430913B0423E0230F0B
:1029A0002D3758F50196A11DB11D20933B0480934E
:1029B0003C0490933D04A0933E04B0933F04809167
:1029C000400490914104A0914204B09143040196C7
:1029D000A11DB11D8093400490934104A093420433
:1029E000B0934304BF91AF919F918F913F912F91ED
:1029F0000F900FBE0F901F90189526E8230F029698
:102A0000A11DB11DD2CF1F920F920FB60F921124AC
:102A10002F938F939F93EF93FF9380916F008B7F02
:102A200080936F00809181008F7B809381008091E3
:102A300050042091EA0320589091E903893020F452
:102A40009695922B8F5FFACF9093E90380914F0474
:102A50008F5F803508F080E020914E04281739F010
:102A6000E82FF0E0E551FC4F908380934F041092E3
:102A70005004809181008F7B809381001092EA0343
:102A8000FF91EF919F918F912F910F900FBE0F901B
:102A90001F9018951F920F920FB60F9211242F932B
:102AA0003F934F935F936F937F938F939F93AF93D6
:102AB000BF93EF93FF9380918600909187004091A0
:102AC000EA03209181004423F1F12F7B20938100C0
:102AD0001092EA033091500431113CC0411122C0E0
:102AE0002091510430915204280F391F30938B00EC
:102AF00020938A0024E026BB20916F00246020935D
:102B00006F002091530430915404820F931F369527
:102B10002795280F391F3093E8032093E70381E0BE
:102B200080935004FF91EF91BF91AF919F918F914E
:102B30007F916F915F914F913F912F910F900FBEB9
:102B40000F901F90189520642093810020E8209317
:102B5000EA03C0CF4091E7035091E803609153042A
:102B600070915404DB01A095B095E091EA032091A7
:102B7000E903841B950BA817B90768F126952E2B3E
:102B8000460F571F3F5F861B970B3930A0F32093EA
:102B9000E90380916F008B7F80936F0080914F04D9
:102BA0008F5F803508F080E090914E04981749F0CF
:102BB000E82FF0E09091E903E551FC4F908380937A
:102BC0004F04809181008F7B809381001092EA03F3
:102BD00010925004A7CF2093E9035093E803409349
:102BE000E703309350049ECF1F920F920FB60F92BF
:102BF00011242F933F934F935F936F937F938F9302
:102C00009F93EF93FF9320914D046091E603809191
:102C10008800909189004091530450915404309160
:102C2000E5032A3070F5840F951F762F71702930D7
:102C300009F471E066952F5F371799F330918000A2
:102C40007723E1F0306C309380009093890080937B
:102C500088007093E5036093E60320934D04FF9191
:102C6000EF919F918F917F916F915F914F913F91E4
:102C70002F910F900FBE0F901F9018953F7B3068DB
:102C8000E2CF30914C04E0914B043E1319C02A303E
:102C900051F42BE020934D04840F951F90938900ED
:102CA00080938800DCCF10924D04809180008F7358
:102CB0008093800080916F008D7F80936F00CFCFD5
:102CC000EF5FE43408F0E0E0E0934B04F0E0EF5510
:102CD000FC4F30813093E6031092E5033091800081
:102CE0003F7B3068309380002A3071F42091530488
:102CF00030915404820F931F909389008093880031
:102D000081E080934D04ABCF809184009091850049
:102D10004096F2CFCF93DF93EC01862F68837983BF
:102D20001A821B821C821D821E821F8218861986AF
:102D30001B861A8662E00E947B0388810E9424031E
:102D40009D878C879F878E87998B888B1A8A1B8A91
:102D50001C8A1D8ADF91CF910895EBE7F6E013827C
:102D6000128288EE93E0A0E0B0E084839583A6838E
:102D7000B7832CE031E03183208325EC30E03587C8
:102D8000248724EC30E03787268720EC30E0318B35
:102D9000208B21EC30E0338B228B22EC30E0358B22
:102DA000248B26EC30E0378B268B118E128E138EFF
:102DB000148EECE2F8E01382128284839583A6835A
:102DC000B7838EE191E091838083F0932B08E093A9
:102DD0002A08EAE5F7E01182108213821282158236
:102DE0001482178216821186108613861286158623
:102DF000148617861686118A108A138A128A158AF3
:102E0000148A178A168A118E108E138E128E158EC2
:102E1000148E178E168E11A210A213A212A215A242
:102E200014A217A216A211A610A68AE298E093A7F0
:102E300082A714A615A616A613AA12AA15AA14AA42
:102E40008FEF9FEF97AB86AB91AF80AF83E080931E
:102E5000940713AE14AE15AE16AE10921908E9E938
:102E6000F7E080E8DF011D928A95E9F710921C08CF
:102E700010921D0810921E0810921F081092200830
:102E80001092210810922208109223081092240810
:102E900010922508109226081092270810922808F0
:102EA0001092290862E070E084E497E00E948A169C
:102EB00063E070E08EE297E00E948A1664E070E0C2
:102EC00088E197E00C948A16CF93DF931F92CDB7D9
:102ED000DEB7789484B5826084BD84B5816084BD9A
:102EE00085B5826085BD85B5816085BD80916E00A8
:102EF000816080936E0010928100809181008260D9
:102F00008093810080918100816080938100809115
:102F100080008160809380008091B1008460809304
:102F2000B1008091B00081608093B00080917A0000
:102F3000846080937A0080917A00826080937A0026
:102F400080917A00816080937A0080917A00806815
:102F500080937A001092C1008FEF93E00E941613C5
:102F60008F3F39F461E08FEF93E00E942C0E0E94B6
:102F7000B812E0918B06F0918C0682E08083E0919C
:102F80008706F09188061082E0918906F0918A0602
:102F90008FEC808310929306E0918F06F09190065B
:102FA00086E08083E0918D06F0918E0680818061BD
:102FB0008083E0918D06F0918E0680818860808309
:102FC000E0918D06F0918E06808180688083E0918B
:102FD0008D06F0918E0680818F7D808390E080E069
:102FE0000E94161390E090934F0680934E0681E066
:102FF00090E00E9416138093030182E090E00E940B
:10300000161380934A048AE090E00E94161380937E
:1030100049048BE090E00E94161391E0811101C0F9
:1030200090E0909348048CE090E00E94161391E0A9
:10303000811101C090E0909347048DE090E00E94E0
:10304000161391E0811101C090E09093460484E151
:1030500090E00E9416132AE0829FC00111249093F1
:103060005906809358068EE190E00E9416138093D3
:1030700045048FE190E00E94161391E0811101C098
:1030800090E09093440461E08EE00E947B0361E055
:103090008FE00E947B0361E080E10E947B0361E09E
:1030A00085E00E947B0361E086E00E947B0361E093
:1030B0008BE00E947B0364E670E080E090E00E9479
:1030C000390484E00E942403019761F483E00E94A4
:1030D0002403892B39F482E00E942403019711F420
:1030E0000E94B81280914E0690914F068230910551
:1030F00009F406C208F0F5C1009709F4FBC1019775
:1031000009F4FBC18091040190910501A091060191
:10311000B09107018093500690935106A0935206F8
:10312000B093530680E596E00E943C0510926F0034
:103130001092800081E88093810080E092E090937B
:1031400054048093530480E892E190935204809356
:10315000510462E088E00E947B0361E089E00E9404
:103160004D0361E089E00E947B03109250041092AD
:103170004F0410924E0410924D0410924C04109281
:103180004B0480E286BB80936F00109286071092FA
:1031900088071092870710928F0710928E0710925F
:1031A0008D0710928C078FEF9FEF9093910780937C
:1031B000900790939307809392070E946B0460930B
:1031C0001C0870931D0880931E0890931F0810928E
:1031D000190810929607109295071092970710926F
:1031E000980710921B0810921A088091940781701A
:1031F000826081608093940788EA9AE090936507E3
:103200008093640789E792E190936707809366074C
:1032100084E19BE0909377078093760784E190E0C8
:10322000A0E0B0E08093460790934707A09348073B
:10323000B09349078093300790933107A0933207EA
:10324000B093330780931A0790931B07A0931C0732
:10325000B0931D0787EE95E017E5C12E14E0D12E3F
:10326000D60111961C921E9213961C921E921297D2
:10327000B4E0CB0ED11C8C159D0591F78EE698E03D
:10328000909344068093430689E698E09093560411
:103290008093550481E0809345066DE871E086E3F4
:1032A0009DE00E94F60560E871E083E193E10E94F1
:1032B000F6056BE771E08BE89DE00E94F60566E796
:1032C00071E08CE294E10E94F60565E671E089EF19
:1032D00093E10E94F60562E571E086EC93E10E94BD
:1032E000F60566E471E089E693E10E94F60568E37D
:1032F00071E081E493E10E94F60565E271E088E106
:1033000093E10E94F60564E171E083E993E10E9494
:10331000F60511E0B0E82B2E312CE0E86E2EF0EF30
:103320007F2E44244394512C84E497E00E94770438
:103330008EE297E00E94770488E197E00E9477048C
:1033400040915007509151072091520730915307F7
:103350004130510521F481E02115310509F080E06B
:1033600080937A06452B21F491E02130310509F054
:1033700090E09093790691E0232B09F090E09093F0
:10338000780640913A0750913B0720913C073091D5
:103390003D074130510521F491E02115310509F037
:1033A00090E090937706452B21F491E02130310590
:1033B00009F090E09093760691E0232B09F090E0DD
:1033C0009093750640912407509125072091260778
:1033D000309127074130510521F491E02115310545
:1033E00009F090E090937406452B21F491E0213090
:1033F000310509F090E09093730691E0232B09F0DA
:1034000090E090937206882379F0109371060E94E1
:103410006B0460936D0670936E0680936F069093B5
:10342000700689E10E94CB0F80917706882379F09E
:1034300010936C060E946B04609368067093690693
:1034400080936A0690936B068AE10E94CB0F80916D
:103450007406882379F0109367060E946B046093CA
:1034600063067093640680936506909366068BE10D
:103470000E94CB0F9091710630916C0620916706E7
:1034800080916206911142C0311151C0222359F03E
:10349000311110935E06911110936006882309F490
:1034A000F3C310935C06882309F4EFC32111109332
:1034B0005C06332309F4E5C310935D06992309F4F0
:1034C00070C710935F06332309F4E1C3222309F484
:1034D000DEC310935B06882309F4D9C310935A0600
:1034E000D6C38330910579F0049709F00BCE0E9482
:1034F000C40E08CE0E941E0F05CE0E94000F02CE01
:103500000E94E20EFFCD0E94A80FFCCD3111109356
:103510006106211110936006882309F4B5CF10933A
:103520005F06332309F4B2CF1093610602C09111F4
:10353000FBCF211110935E06882309F4A7CF1093C7
:103540005D06A4CF8B3109F4F7C08F3709F00EC7A1
:1035500087E0F0C0E0914106F0914206E550FA4F55
:10356000108285EF92E00E94E705EBEFF5E0019015
:103570000020E9F79F012B5F35408BEF95E090939A
:10358000E8058093E70560E0F12CE12C70E090E025
:1035900080E0FC01E550FA4F4081403209F46EC0F2
:1035A0002CF4442309F452C060E006C0423209F40E
:1035B00052C0602F4C35C1F701968217930724F44F
:1035C000BAE0EB16F10429F790E0E92FF0E0EE15F0
:1035D000FF050CF464C037E5A32E34E0B32ED5010B
:1035E0008D909C9011978114910489F012966D91A1
:1035F0007C918091E7059091E8050E941022892B2B
:1036000031F467EE75E0C701F401099500E0F4E0DC
:10361000AF0EB11CCA14DB0411F7002371F08091C6
:10362000410690914206892B41F08BE991E00E947E
:10363000D90588E991E00E94D905109242061092BE
:10364000410685EF92E00E94E70576C09FEFE91AF8
:10365000F90AC901A9CF6111A7CF108271110CC05D
:10366000F701EE0FFF1FE951FA4FAC0144505A4FDA
:103670005183408371E0A0CF70E09ECF711194CF51
:103680001082AFEFEA1AFA0AF701EE0FFF1FE951B5
:10369000FA4FAC0144505A4F5183408385CFEE0F0F
:1036A000FF1FE951FA4F20813181D9010D9000208F
:1036B000E9F711975D01A21AB30A80E060E0262FB6
:1036C00030E02A153B0514F09F5F7FCF4081518188
:1036D000D901A80FB11DA40FB51F7C917C3549F409
:1036E00011967C91723229F4420F531FDA017C93B8
:1036F0008F5F882351F040815181240F351FD901FC
:10370000A80FB11D4C91D9014C936F5FD8CF809118
:10371000410690914206009709F41ACF01979093C1
:1037200042068093410688E00E94A10580E20E9443
:10373000A10588E00E94A105B090860720E12B1525
:1037400008F47AC0E0918407F09185078081918127
:10375000DC01ED91FC910084F185E02D0995892B28
:1037600009F46AC0809129088E7F80932908E0912E
:103770008407F091850780819181DC01ED91FC91B6
:103780000284F385E02D0995082F8D3F09F454C07C
:1037900080918E0790918F07009709F01FC10093C9
:1037A0008907F09087078F2D0E9417060E94250633
:1037B000882351F007FD08C0F092890700938A071B
:1037C00050928F0740928E0700918907802F0E94A8
:1037D0001706813F09F4CDC008F066C0803B39F080
:1037E00068F4803921F0803A11F0803879F423E0D0
:1037F00030E030938D0720938C07C1C0803D09F4E1
:10380000B8C008F042C0803C09F4B3C080912908D8
:10381000816080932908E0915C07F0915D07309703
:1038200009F0099510928F0710928E0710928D075C
:1038300010928C071092870780E596E00E9412058F
:10384000882341F080914E0690914F06069711F023
:103850000E94BB0786E496E00E941205882341F08F
:1038600080914E0690914F06069711F40E94CE0863
:1038700020E030E0232B09F457CD0E945802882322
:1038800009F44BCD0E94000048CD803E09F4AFCF33
:10389000803F09F0BBCF30928D0720928C071092A9
:1038A0008707809399076BC0873FA9F308F05AC038
:1038B000833F09F45EC008F49ACF863F09F0A6CF93
:1038C0008093960710929507109297071092980789
:1038D0001093190810928F0710928E0710928D077F
:1038E00010928C0780919607803931F48091980767
:1038F000811102C0609296078091960780588136A8
:1039000030F480919507B81611F0B11002C00E94F2
:10391000080190919407392F317090FF8DCF892F36
:103920008E7F09F489CF8091960720E8280F2136F1
:1039300008F01FC120919507B21619F031E0B110BF
:1039400030E09695923009F40DC1933009F40EC120
:10395000913009F071CF40919807609197070E94CC
:103960007F066ACF8D3F08F4ABCF8E3F08F0A8CF1B
:103970004DCFE2E0F0E0F0938D07E0938C072091CB
:103980008E0730918F0740918C0750918D074150E1
:10399000510924173507D8F0809396070F700F5FF1
:1039A0000093950780918A07809397071092980754
:1039B00050921B0840921A0810928F0710928E079F
:1039C00010928D0710928C07109319088BCF2F5FE0
:1039D0003F4F30938F0720938E072ECF07FF0CC0E9
:1039E0000D3F08F043C0083F08F042C0003F09F413
:1039F0004CC0073F09F449C020918907FC01E65AF1
:103A0000F84F203F19F0273F09F067C007AFE0905B
:103A10008C07F0908D079701215031098217930789
:103A200008F49AC0A0908907B0EFAB1619F0E7EF41
:103A3000AE1255C00091180870921808709296073F
:103A400060929707109298071092950730921B0882
:103A500020921A08109319080E940801F7EFF093BA
:103A6000990700939A0722E030E0B3CF0E3F20F28F
:103A70000093960710929707109298071092950757
:103A800050921B0840921A089FCF20919907203F1F
:103A900019F0273F09F0BACE9C012F5F3F4F865A9D
:103AA000984FDC01DF960C9370929607209397074E
:103AB000309398071092950730931B0820931A08AB
:103AC0001093190810928F0710928E0710928D078D
:103AD00010928C071092870705CF07A798CF8A2DE1
:103AE0000E941706082F809396070E9425068823B8
:103AF00041F18A2D8F708F5F8093950780918A079F
:103B00008093970780918B0733E0E316F10409F067
:103B100080E08093980710928F0710928E07109282
:103B20008D0710928C0710931908003B39F060F450
:103B3000003921F0003A11F0003861F6A0928707B1
:103B4000D1CE10929507DACF003DC1F3003EB1F31C
:103B5000003C09F0BFCFF2CF019690938F0780937E
:103B60008E076ACE332309F467CEF5CE311164CEC9
:103B7000F2CEE0E1E80FE03108F05ECEF0E0ED5388
:103B8000F24E0C94BA24D91D2D1E0E1EFC1D1C1CB9
:103B90001C1CD31D1C1CD31D1C1CD31DD31DD31DCD
:103BA0001C1CD31DD31D682F84E897E00E9471066A
:103BB00043CEA0909707B090980741E8A416B104AF
:103BC00018F020E8A22EB12C9AE5E92E97E0F92E04
:103BD000C7018A5597408A159B0508F02DCED7015D
:103BE000DF966C9180918407909185070E9434063E
:103BF000BFEFEB1AFB0AECCF0091970763EF8091C0
:103C00008407909185070E943406602F6F7780911A
:103C10008407909185070E9434060ECEE0909807A5
:103C2000E0E8EE9E7001112480919707E82A62EF88
:103C300080918407909185070E9434066E2D6F77DE
:103C400080918407909185070E943406B701660F22
:103C5000672F661F770B7195D9CF80919707F0E199
:103C60008F9FC00111248077009198070F70082B57
:103C700061EF80918407909185070E943406602F40
:103C8000C6CF91111ECC03C080E091111CCC809155
:103C900079068823B9F09923A9F0809161068111F2
:103CA00011C08091600681110DC080915B06811169
:103CB00009C080915F06811105C081E00E94CB0F91
:103CC0000E946807809176068823E9F080916C064F
:103CD0008823C9F080916106811115C080915E062C
:103CE000811111C080915D0681110DC080915B062C
:103CF000811109C080915A06811105C082E00E949D
:103D0000CB0F0E946807809173068823E9F08091A9
:103D100067068823C9F080915E06811115C08091E5
:103D20005C06811111C08091600681110DC08091E7
:103D30005A06811109C080915B06811105C083E09C
:103D40000E94CB0F0E94680780917906811104C000
:103D5000809176068823E9F0809171068823C9F066
:103D600080916C068823A9F080916106882389F0F0
:103D700080915B0681110DC080916006811109C0A0
:103D800080915F06811105C085E00E94CB0F0E94E3
:103D9000680780917906811104C080917306882399
:103DA000C9F0809171068823A9F080916706882365
:103DB00089F080916006882369F080915B0681110B
:103DC00009C080916106811105C086E00E94CB0F79
:103DD0000E94680780917606811104C08091730665
:103DE000882309F180916C068823E9F080916706A9
:103DF0008823C9F080915E068823A9F080915B0634
:103E0000811111C080915A0681110DC08091600608
:103E1000811109C080915D06811105C087E00E9473
:103E2000CB0F0E94680780917606882309F1809164
:103E30006C068823E9F0809162068823C9F080919E
:103E40005D068823A9F080915B06811111C08091E5
:103E50005A0681110DC080916106811109C08091BF
:103E60005C06811105C088E00E94CB0F0E946807A4
:103E700080917306882329F180916706882309F1D0
:103E8000809162068823E9F080915C068823C9F05E
:103E900080915B06811115C080915A06811111C075
:103EA0008091600681110DC080915D06811109C06D
:103EB00080915F06811105C089E00E94CB0F0E94AE
:103EC000680780917906882309F18091710688231B
:103ED000E9F0809162068823C9F080915F0688230B
:103EE000A9F080915B06811111C08091610681115A
:103EF0000DC080915C06811109C080915A06811124
:103F000005C082E10E94CB0F0E946807809179066C
:103F1000811108C080917606811104C080917306DA
:103F20008823A9F080917106882389F080916C061E
:103F3000882369F080916706882349F080915B06A9
:103F4000882329F08AE00E94CB0F0E9468078091A5
:103F50007606811104C0809173068823A9F08091B0
:103F60006C06882389F080916706882369F0809128
:103F70006206882349F080915A06882329F08BE055
:103F80000E94CB0F0E94680780917106882371F10F
:103F900080917806882351F10E946B0480906D0611
:103FA00090906E06A0906F06B0907006AB01BC01B9
:103FB000481959096A097B09809158069091590658
:103FC000092E000CAA0BBB0B84179507A607B70791
:103FD00068F480917506811109C080917206811183
:103FE00005C00E9468078CE00E94CB0F80916C0690
:103FF000882371F180917506882351F10E946B042A
:104000008090680690906906A0906A06B0906B0652
:10401000AB01BC01481959096A097B09809158060E
:1040200090915906092E000CAA0BBB0B841795071B
:10403000A607B70768F480917806811109C08091BE
:104040007206811105C00E9468078DE00E94CB0FA7
:1040500080916706882371F180917206882351F15F
:104060000E946B048090630690906406A0906506A1
:10407000B0906606AB01BC01481959096A097B0971
:104080008091580690915906092E000CAA0BBB0B83
:1040900084179507A607B70768F480917806811101
:1040A00009C080917506811105C00E9468078EE0E5
:1040B0000E94CB0F80917106882309F48EC08091F5
:1040C0006C06882309F445C080917806882309F49A
:1040D00040C0809175068823E1F1809172068111BC
:1040E00038C00E946B048090580690905906092CA5
:1040F000000CAA08BB0820916D0630916E06409115
:104100006F0650917006621B730B840B950B86161D
:104110009706A806B906E8F40E946B042091680689
:104120003091690640916A0650916B06621B730BD1
:10413000840B950B86169706A806B90650F40E94C4
:10414000680780E10E94CB0F80917106882309F4F3
:1041500044C080916706882309F43FC080917806A7
:104160008823D9F1809172068823B9F18091750670
:10417000811133C00E946B048090580690905906BC
:10418000092C000CAA08BB0820916D0630916E0620
:1041900040916F0650917006621B730B840B950B58
:1041A00086169706A806B906C0F40E946B042091F3
:1041B0006306309164064091650650916606621B65
:1041C000730B840B950B86169706A806B90628F480
:1041D0000E94680781E10E94CB0F80916C068823C2
:1041E00009F444C080916706882309F43FC0809198
:1041F00075068823D9F1809172068823B9F18091E0
:104200007806811133C00E946B048090580690900C
:104210005906092C000CAA08BB08209168063091A9
:10422000690640916A0650916B06621B730B840B02
:10423000950B86169706A806B906C0F40E946B0473
:1042400020916306309164064091650650916606A0
:10425000621B730B840B950B86169706A806B9068E
:1042600028F40E94680784E10E94CB0F80917106B8
:10427000882309F45FC080916C06882309F45AC032
:1042800080916706882309F455C0809178068823B9
:1042900009F450C080917506882309F44BC08091C1
:1042A0007206882309F446C00E946B048090580669
:1042B00090905906092C000CAA08BB0820916D06A5
:1042C00030916E0640916F0650917006621B730B21
:1042D000840B950B86169706A806B90658F50E941A
:1042E0006B04209168063091690640916A065091EE
:1042F0006B06621B730B840B950B86169706A8063C
:10430000B906C0F40E946B042091630630916406E4
:104310004091650650916606621B730B840B950BEA
:1043200086169706A806B90628F40E94680787E152
:104330000E94CB0F198200914506002309F4FCC9A5
:10434000E0914306F0914406CE0101960995892B30
:1043500009F4F2C989818D3009F4FCC80CF0F2C867
:10436000883009F4D4C9893009F4F2C82091410693
:10437000309142062534310508F0DEC980320CF454
:10438000DBC925503A4FF90180830E94A105809135
:104390004106909142060196909342068093410611
:1043A000CBC921119BC873CC8EE191E090932D086D
:1043B00080932C0880916F008B7F80936F00809199
:1043C0006F008F7D80936F0080914E0480934F0427
:1043D00080914D048111FCCF80916F008D7F80937F
:1043E0006F000895FC0188279927E89421912032D5
:1043F000E9F3293010F02E30C8F32B3241F02D3282
:1044000039F4689404C00E941922820F911D2191F1
:1044100020532A30C0F31EF4909581959F4F089544
:10442000FB01DC018D91059080190110D9F3990BE6
:1044300008957AE0979F902D879F802D910D1124EC
:104440000895F999FECF92BD81BDF89A992780B55C
:104450000895262FF999FECF1FBA92BD81BD20BDC8
:104460000FB6F894FA9AF99A0FBE0196089550582B
:10447000BB27AA270E944F220C94A0230E949223BC
:1044800038F00E94992320F039F49F3F19F426F464
:104490000C948F230EF4E095E7FB0C948923E92F0D
:1044A0000E94B12358F3BA17620773078407950770
:1044B00020F079F4A6F50C94D3230EF4E0950B2E9E
:1044C000BA2FA02D0B01B90190010C01CA01A00166
:1044D0001124FF27591B99F0593F50F4503E68F1C1
:1044E0001A16F040A22F232F342F4427585FF3CF02
:1044F000469537952795A795F0405395C9F77EF4D3
:104500001F16BA0B620B730B840BBAF09150A1F01B
:10451000FF0FBB1F661F771F881FC2F70EC0BA0FA1
:10452000621F731F841F48F4879577956795B79529
:10453000F7959E3F08F0B0CF9395880F08F0992724
:10454000EE0F9795879508950E94B8220C94A023AA
:104550000E94992358F00E94922340F029F45F3F73
:1045600029F00C94892351110C94D4230C948F239B
:104570000E94B12368F39923B1F3552391F3951B5E
:10458000550BBB27AA2762177307840738F09F5F74
:104590005F4F220F331F441FAA1FA9F335D00E2EE1
:1045A0003AF0E0E832D091505040E695001CCAF74E
:1045B0002BD0FE2F29D0660F771F881FBB1F261711
:1045C00037074807AB07B0E809F0BB0B802DBF01E8
:1045D000FF2793585F4F3AF09E3F510578F00C94B7
:1045E00089230C94D4235F3FE4F3983ED4F386955B
:1045F00077956795B795F7959F5FC9F7880F911DD8
:104600009695879597F90895E1E0660F771F881FC3
:10461000BB1F621773078407BA0720F0621B730B76
:10462000840BBA0BEE1F88F7E09508950E941D23B6
:104630006894B1110C94D42308950E94B92388F092
:104640009F5798F0B92F9927B751B0F0E1F0660F56
:10465000771F881F991F1AF0BA95C9F714C0B13097
:1046600091F00E94D323B1E008950C94D323672FD7
:10467000782F8827B85F39F0B93FCCF386957795C6
:104680006795B395D9F73EF49095809570956195AF
:104690007F4F8F4F9F4F0895E89409C097FB3EF4DA
:1046A00090958095709561957F4F8F4F9F4F99237F
:1046B000A9F0F92F96E9BB279395F69587957795FD
:1046C0006795B795F111F8CFFAF4BB0F11F460FFBD
:1046D0001BC06F5F7F4F8F4F9F4F16C0882311F015
:1046E00096E911C0772321F09EE8872F762F05C029
:1046F000662371F096E8862F70E060E02AF09A95C4
:10470000660F771F881FDAF7880F9695879597F9B8
:10471000089597F99F6780E870E060E008959FEF43
:1047200080EC089500240A94161617061806090648
:10473000089500240A941216130614060506089517
:10474000092E0394000C11F4882352F0BB0F40F49F
:10475000BF2B11F460FF04C06F5F7F4F8F4F9F4FDF
:10476000089557FD9058440F551F59F05F3F71F061
:104770004795880F97FB991F61F09F3F79F08795C8
:104780000895121613061406551FF2CF4695F1DF51
:1047900008C0161617061806991FF1CF86957105E1
:1047A000610508940895E894BB2766277727CB0115
:1047B00097F908950E944C2408F48FEF08950E9401
:1047C000F2230C94A0230E94922338F00E94992394
:1047D00020F0952311F00C9489230C948F2311243D
:1047E0000C94D4230E94B12370F3959FC1F3950FCD
:1047F00050E0551F629FF001729FBB27F00DB11D65
:10480000639FAA27F00DB11DAA1F649F6627B00DF4
:10481000A11D661F829F2227B00DA11D621F739FDD
:10482000B00DA11D621F839FA00D611D221F749FEB
:104830003327A00D611D231F849F600D211D822F32
:10484000762F6A2F11249F5750409AF0F1F0882359
:104850004AF0EE0FFF1FBB1F661F771F881F915086
:104860005040A9F79E3F510580F00C9489230C9489
:10487000D4235F3FE4F3983ED4F38695779567950C
:10488000B795F795E7959F5FC1F7FE2B880F911DB0
:104890009695879597F90895990F0008550FAA0BDB
:1048A000E0E8FEEF16161706E807F907C0F0121643
:1048B0001306E407F50798F0621B730B840B950B46
:1048C00039F40A2661F0232B242B252B21F408959B
:1048D0000A2609F4A140A6958FEF811D811D089538
:1048E000AA1BBB1B51E107C0AA1FBB1FA617B70716
:1048F00010F0A61BB70B881F991F5A95A9F7809532
:104900009095BC01CD01089597FB072E16F40094F5
:1049100007D077FD09D00E94702407FC05D03EF433
:10492000909581959F4F0895709561957F4F08955B
:10493000A1E21A2EAA1BBB1BFD010DC0AA1FBB1FA3
:10494000EE1FFF1FA217B307E407F50720F0A21B15
:10495000B30BE40BF50B661F771F881F991F1A9482
:1049600069F760957095809590959B01AC01BD01AC
:10497000CF010895EE0FFF1F0590F491E02D0994EB
:1049800010E0CDEDD0E004C0FE010E94BA242196D3
:0A499000CE3DD107C9F7F894FFCF20
:10499A00FFFF01012C010000000000008E02EE0161
:1049AA001B02DB024C022A023E02000000009208AF
:1049BA00EE01CB088D08D904FC04E9042D2D2D2D18
:1049CA002D2D2D2D2D2D2D2D2D2D2D2D2D2D2D2D0D
:1049DA002D2D2D2D2D2D2D2D2D0D0A006D6964697E
:1049EA006368616E6E656C203D2025640D0A007453
:1049FA00687275203D2025640D0A00707265736522
:104A0A0074746170656E61626C6564203D20256412
:104A1A000D0A00736E617073686F74746170656EED
:104A2A0061626C6564203D2025640D0A0065786921
:104A3A007474756E6572616E79627574746F6E20C6
:104A4A003D2025640D0A006C6F6E67707265737382
:104A5A0074696D656F7574203D2025640D0A0054D4
:104A6A007269706C6520492F4F206669726D776193
:104A7A00726520762E20342E3031006B676D6964A2
:104A8A0069636F6E74726F6C6C6572732E636F6D8F
:104A9A000D0A00417661696C61626C6520636F6D15
:104AAA006D616E64733A0D0A0073686F7776616C94
:104ABA007565730D0A006D6964696368616E6E6578
:104ACA006C2028312D3136290D0A00746872752040
:104ADA0028302F31290D0A006C6F6E67707265736A
:104AEA007374696D656F757420283230302D3235D4
:104AFA003030290D0A0070726573657474617065CF
:104B0A006E61626C65642028302F31290D0A0065B8
:104B1A0078697474756E6572616E79627574746F92
:104B2A006E2028302F31290D0A00736E6170736868
:104B3A006F74746170656E61626C65642028302FD1
:104B4A0031290D0A00666163746F72797265736543
:104B5A00740D0A004572726F722E2057726F6E675B
:104B6A0020636F6D6D616E64206F7220617267756C
:104B7A006D656E742072616E67652E200D0A004F96
:104B8A004B2E200D0A007072657365743A202564F5
:104B9A002C2072696E67746F626C696E6B3A20259D
:104BAA00640D0A0062616E6B206368616E6765203E
:104BBA0063616E63656C6C65640062616E6B203D57
:104BCA002025640062616E6B3A2025640D0A006D2F
:104BDA006F6465203D2000736E617073686F746244
:104BEA00746E70726573736564203D2025640D0AC6
:104BFA00002564206D696C697365636F6E64730D5B
:024C0A000A009E
:00000001FF
